:020000040000FA
:0600000060283F300130D2
:08000800A000030EA100831209
:1000100005191028831601178312B2308100422877
:100020008316011383120B191C28AE17280A031913
:100030002E17AE192D283B28AE13AE192A282E1FD5
:100040003B28AE1A3B28A701A601A501A801AE01D5
:10005000AE164228F030AE0542282D152E13AE12F2
:100060002708AB002608AA002508A9002808AC002C
:10007000F030AE0542282E0DA80DA50DA60DA70D3A
:10008000AE1AAE0A8B100B11210E8300A00E200EAB
:02009000090065
:1000C000203084008001840A60300402031C62280E
:1000D000F3218316FF239000831283160C308505CD
:1000E000870183128501870107309900003083164C
:1000F00091009F008312C830831681008312313033
:100100009000003083168C00831210308B003D1B52
:10011000BE013D1BBF013D1F1E2281018E018F01CB
:100120000B118B100B108C130C138C110C108B17E4
:10013000A8202D19AA20C721B30BA62803108519C2
:100140000314BA0DF0303A0203193F211F229828F8
:1001500064000800A91F2D11A91F0800291B2D11DB
:10016000291B08002B082A0629062C02031D2D1125
:10017000031D08002D110130B7008B132030370705
:1001800083169B001C141A088312A4001030370732
:1001900083169B001C141A088312A3000030370733
:1001A00083169B001C141A088312A2008B172408C4
:1001B0002B02031D392923082A02031D392922088D
:1001C0002906F039A91EE039031D3929220829051D
:1001D0000F3903190F2901303702031DF4283E1887
:1001E000F4283E14AD17022202303702031DFD2809
:1001F000BE18FD28BE14AD17052203303702031DBB
:1002000006293E1906293E15AD170822043037028B
:10021000031D0F29BE190F29BE15AD170B22290981
:1002200022050F390319392901303702031D1D2911
:100230003E1C1D293E10AD170E2202303702031D51
:100240002629BE1C2629BE10AD1712220330370204
:10025000031D2F293E1D2F293E11AD1716220430F4
:100260003702031D3829BE1D3829BE11AD171A22C9
:100270003929B70A0530370203180800BD28B6012E
:10028000B3019630B4000130B5000130B7008501EC
:100290008701AD13A721A820B30B68290310851986
:1002A0000314BA0DF0303A0203199729B41F8501DF
:1002B000B41F8701B40B68293708B6080319B600C4
:1002C00003196629FF3085008700B6039630B40015
:1002D0002D1D4B292D11A91F4B29291B4B29A91E67
:1002E00029120F30290503194B29B9012918B90A18
:1002F000A918B90A2919B90AA919B90AB9184B29AB
:1003000039194B298B1320303707BC002B08BB0051
:10031000D52110303707BC002A08BB00D52100309A
:100320003707BC002908BB00D5218B17A121850107
:100330008701B70AB60105303702031C4B291E227C
:1003400008000430370203190800850187011430C2
:10035000B90033300F1E85000F1A8501FF300F1AC8
:1003600087000F1E8701A8202D1DA9292D11290AFC
:100370000319BE29A91FA929291BA9290F3029055D
:10038000031DA729B90BA929850187010800AD1F05
:100390000800AD131030BC003E08BB00D521303042
:1003A000BC003F08BB00D52108003C088B13831616
:1003B0009B001C141A0883128B173B0203190800B8
:1003C0008B133B0883161C159A003C089B00553084
:1003D0009D00AA309D009C1464009C18EC291C11FF
:1003E00083128B170800831600309B001C141A0818
:1003F0008312BD00831610309B001C141A08831250
:10040000BE0008000130BE0008000230BE00080037
:100410000430BE0008000830BE00080085018701D6
:100420003E10080085018701BE1008008501870184
:100430003E11080085018701BE11080008008F08E1
:10044000031908008F0103303E050319172B0230F2
:100450003E05031D51105408EB3C031805125118BA
:10046000342AD40B3F2A392AD4035408C83C031C2D
:100470003F2A0516F530D4005108013AD100023068
:100480003E05031DD1105508E63C03188512D1180E
:100490004C2AD50B572A512AD5035508B93C031CC1
:1004A000572A8516F030D5005108023AD1000230A3
:1004B0003E05031D51115608DC3C03180510511967
:1004C000642AD60B6F2A692AD6035608B63C031C49
:1004D0006F2A0514E630D6005108043AD1000230E4
:1004E0003E05031DD1115708F03C03188510D119A2
:1004F0007C2AD70B872A812AD7035708D73C031CAD
:10050000872A8514FA30D7005108083AD100023002
:100510003E05031D51125808E03C03188710511A7C
:10052000942AD80B9F2A992AD8035808C13C031C47
:100530009F2A8714EA30D8005108103AD1000630BB
:100540003E05031DD1125908D43C03180711D11AD6
:10055000AC2AD90BB72AB12AD9035908A73C031CE6
:10056000B72A0715DE30D9005108203AD1000630ED
:100570003E05031D51135A08BF3C03180710511BB9
:10058000C42ADA0BCF2AC92ADA035A089C3C031C76
:10059000CF2A0714C930DA005108403AD10006309A
:1005A0003E05031DD1135B08D73C03188712D11BEE
:1005B000DC2ADB0BE72AE12ADB035B08BE3C031CD9
:1005C000E72A8716E130DB005108803AD100063077
:1005D0003E05031D52105C08F13C03180712521827
:1005E000F42ADC0BFF2AF92ADC035C08CF3C031C4D
:1005F000FF2A0716FB30DC005208013AD200063011
:100600003E05031DD2105D08E93C03188711D2187E
:100610000C2BDD0B172B112BDD035D08B23C031CEB
:10062000172B8715F330DD005208023AD2000C3048
:100630003E050319672B3E1D232B54083C3C031C2D
:10064000232B85018701D40B0800D0034630D4004A
:100650000B305002031D2D2B05160A305002031DCE
:10066000322B851609305002031D372B0514083034
:100670005002031D3C2B851407305002031D412BF3
:10068000871406305002031D462B07150530500213
:10069000031D4B2B071404305002031D502B8716EB
:1006A00003305002031D552B071602305002031D64
:1006B0005A2B871501305002031D5E2B1230500259
:1006C000031C0800850187010C30D0000800203091
:1006D0003E050319B12BD40B722B0508103A850087
:1006E0008230D400D50B792B0508203A85007D3067
:1006F000D500D60B802B0508013A85007330D60053
:10070000D70B872B0508023A85008730D700D80B16
:100710008E2B0708023A87007730D800D90B952B2B
:100720000708043A87006B30D900DA0B9C2B0708C6
:10073000013A87005630DA00DB0BA32B0708203A7A
:1007400087006E30DB00DC0BAA2B0708103A87000D
:100750008830DC00DD0BB12B0708083A87008030B9
:10076000DD0040303E050319B72B850187010800E5
:084000000600000006000200AA
:02400E00CC01E3
:1042000001008100820084008800B100B200B40087
:10421000B800A100A200FF00FF00FF00FF00FF00A8
:104220000000010001000100010001000100010087
:10423000010001000100FF00FF00FF00FF00FF0080
:10424000010000000000000000000000000000006D
:10425000000000000000FF00FF00FF00FF00FF0063
:104260000000FF00FF00FF00FF00FF00FF00FF0055
:10427000FF00FF00FF00FF00FF00FF00FF00FF0046
:10428000FF00FF00FF00FF00FF00FF00FF00FF0036
:10429000FF00FF00FF00FF00FF00FF00FF00FF0026
:1042A000FF00FF00FF00FF00FF00FF00FF00FF0016
:1042B000FF00FF00FF00FF00FF00FF00FF00FF0006
:1042C000FF00FF00FF00FF00FF00FF00FF00FF00F6
:1042D000FF00FF00FF00FF00FF00FF00FF00FF00E6
:1042E000FF00FF00FF00FF00FF00FF00FF00FF00D6
:1042F000FF00FF00FF00FF00FF00FF00FF00DD00E8
:00000001FF
